:1000000055AA55AA0200000036700000000000004A
:1000100065220000000000000E100000000000003B
:1000200000000000000000000E100000E861000069
:10003000000800000000000000000000B764BF5C82
:1000400024835B4A79180000DB7CA4B586E7FFFFB8
:1000500000021000E1000000034E0000A1010000BA
:10006000ED010000390200008502000000000000E0
:10007000000000000000000000000000074E00002B
:100080000F4E000000000000D1020000174E0000DB
:100090001F4E00002D4E0000354E0000434E000064
:1000A000514E00005F4E0000674E0000754E00008C
:1000B000C34E0000DF020000834E00008B4E0000A4
:1000C000000000009B4E0000C54E0000C74E00001F
:1000D000D54E0000D74E0000D94E0000B34E0000B0
:1000E000BB4E0000A34E0000AB4E0000DB4E0000F4
:1000F000DD4E0000EB4E0000934E000000000000BB
:1001000000000000000000000000000000000000EF
:100110006522000001000140000000000000000016
:1001200000000000000000000000000000000000CF
:1001300000F002F800F03AF80AA090E8000C8244BF
:100140008344AAF10107DA4501D100F02FF8AFF29C
:10015000090EBAE80F0013F0010F18BFFB1A43F0A5
:1001600001031847785E0000A85E0000103A24BF23
:1001700078C878C1FAD8520724BF30C830C144BF0C
:1001800004680C607047000000230024002500264E
:10019000103A28BF78C1FBD8520728BF30C148BFEA
:1001A0000B6070471FB51FBD10B510BDDFF80CD038
:1001B000FFF7F8FF04F055FF05F06EFB000210009A
:1001C00003B4FFF7F1FF03BC05F06EFB40BA7047C4
:1001D000C0BA704772B6784600F10A004DF8080CB4
:1001E00062B630BF00BF704740BA7047C0BA7047B0
:1001F00011484FF00F0100F8011B4FF0010100F80A
:10020000011B4FF0020100F8011B4FF0000100F844
:10021000011B00F8011B00F8011B00F8011B00F88E
:10022000011B1EF0040F0CBFEFF30880EFF30980F1
:100230004FF0020103F056BD0002002011484FF0BC
:100240000F0100F8011B4FF0010100F8011B4FF0F6
:10025000030100F8011B4FF0000100F8011B00F83A
:10026000011B00F8011B00F8011B00F8011B1EF028
:10027000040F0CBFEFF30880EFF309804FF0030188
:1002800003F030BD0002002011484FF00F0100F8CC
:10029000011B4FF0010100F8011B4FF0040100F8B1
:1002A000011B4FF0000100F8011B00F8011B00F8D2
:1002B000011B00F8011B00F8011B1EF0040F0CBF0E
:1002C000EFF30880EFF309804FF0040103F00ABD5B
:1002D0000002002011484FF00F0100F8011B4FF001
:1002E000010100F8011B4FF0050100F8011B4FF060
:1002F000000100F8011B00F8011B00F8011B00F8C9
:10030000011B00F8011B1EF0040F0CBFEFF3088067
:10031000EFF309804FF0050103F0E4BC0002002078
:1003200000B504F08DFD5DF804EB00F02FB81EF071
:10033000040F0CBFEFF30880EFF309804FF00001CA
:1003400003F0D0BC0A484FF0FF0101704FF00000ED
:1003500080F311884FF0000080F3098805484FF0C2
:100360000201017062B604484FF08051016070478D
:1003700022ED00E00703100004ED00E002484FF01A
:10038000805101607047000004ED00E04FF0200054
:1003900080F31188EFF3098098B112480068124980
:1003A0000968884217D0EFF309800E49096820E9EF
:1003B000F00F886000B50B48006804F026FF5DF878
:1003C00004EB084808490A68026000688168B1E8DF
:1003D000F00F81F309884EF0040E4FF0000080F317
:1003E00011887047080310000C031000EFF3118010
:1003F0004FF0200181F31188704700004FF000009A
:1004000080F311887047000062B6704772B670477B
:1004100010B5022000F00AFA032000F007FA0420C9
:1004200000F004FA052000F001FA062000F0FEF9C1
:10043000072000F0FBF9082000F0F8F9092000F08F
:10044000F5F90F2000F0F2F94FF00051002001F80B
:100450004A0F8871F022CA710F224A70F949086266
:1004600088620863886008618861C8604861C86103
:100470004862C86248630621022000F0F6F90621AE
:10048000032000F0F2F90621042000F0EEF9062125
:10049000052000F0EAF90621084600F0E6F90621F9
:1004A000072000F0E2F90621082000F0DEF904211F
:1004B000092000F0DAF906210F2000F0D6F9022019
:1004C00000F0C8F9032000F0C5F9042000F0C2F9DB
:1004D000052000F0BFF9062000F0BCF9072000F06D
:1004E000B9F9082000F0B6F9092000F0B3F90220AC
:1004F00000F091F9032000F08EF9042000F08BF950
:10050000052000F088F9062000F085F9072000F0AA
:1005100082F9082000F07FF9BDE81040092000F0C2
:100520007AB94FF00051C98C4FEA90100A06C549BC
:1005300001D5C54A00E0C54AB2FBF0F0086070473B
:100540004FF0005090F84A00000700D0012070479B
:100550007047BF4900200860BA498860C86070478A
:10056000B84AD160642148430A2190FBF1F0B0F50C
:10057000803F06DBA0F57F40FF3890604FF6FF70AC
:1005800002E0002180B2916000F07FB9AD4910B562
:100590008868B0F5803F06DBA0F57F40FF388860B3
:1005A0004FF6FF7003E030B10022C0B28A60BDE8B0
:1005B000104000F06AB9CA68FFF7CBFF12B1BDE87E
:1005C000104010470020FFF7C3FF10BDA0490020D6
:1005D000091D08609B49086148617047994A51614B
:1005E000642148430A2190FBF1F0B0F5803F06DB1F
:1005F000A0F57F40FF3810614FF6FF7002E0002148
:1006000080B2116100F04BB98E4910B50869B0F5A0
:10061000803F06DBA0F57F40FF3808614FF6FF7092
:1006200004E0002806DD002280B20A61BDE8104027
:1006300000F035B94A69FFF7C9FF12B1BDE81040B3
:1006400010470120FFF784FF10BD814900200831C9
:1006500008607C498861C86170477A4910B588692B
:10066000B0F5803F06DBA0F57F40FF3888614FF68C
:10067000FF7003E030B1002280B28A61BDE8104013
:1006800000F017B9CA69FFF7E0FF12B1BDE81040EA
:1006900010470220FFF75CFF10BD6D4900201031AC
:1006A00008606849086248627047664910B5086A80
:1006B000B0F5803F06D3A0F57F40FF3808624FF6C3
:1006C000FF7003E030B1002280B20A62BDE8104042
:1006D00000F0F9B84A6AFFF7E0FF12B1BDE8104038
:1006E00010470420FFF734FF10BD59490020143192
:1006F000086054498862C8627047524AD1621168E2
:1007000048430A21B0FBF1F0B0F5803F06DBA0F5CD
:100710007F40FF3890624FF6FF7002E0002180B208
:10072000916200F0DBB84FF00050B0F85A00454934
:10073000096908447047434910B5886AB0F5803F9D
:1007400006D3A0F57F40FF3888624FF6FF7003E0C4
:1007500030B1002280B28A62BDE8104000F0BEB81D
:10076000CA6AFFF7C2FF12B1BDE81040104705206A
:10077000FFF7EEFE10BD4020C10581F82100704753
:10078000334800211C3001604FF000524FF6FF71DA
:10079000A2F866100121016070472D4900201C312C
:1007A000086070474FF0005090F82110C90606D538
:1007B00010F8211F21F01001017001207047002066
:1007C000704710B504460F2000F044F80F2000F0E9
:1007D00022F81C4844604FF00050C18C090602D535
:1007E0004EF6602101E04AF6C871416518490120C2
:1007F000B8310860091D086010BD10B50F2000F069
:1008000015F84FF00050C06C0E4920F07F40496849
:10081000BDE81040084700F01F0201219140400947
:10082000800000F1E020C0F80011704700F01F02C6
:10083000012191404009800000F1E020C0F88011C2
:100840007047000000021000C0270900D0DD06003C
:100850004009002200F01F02012191404009800060
:1008600000F1E020C0F88012EAE74907090E0028ED
:1008700006DA00F00F0000F1E02080F8141DDFE739
:1008800000F1E02080F80014DAE71A4900220A603B
:100890004FF00052A2F8580001200860D0E7154937
:1008A0000022091D0A60CA06A2F85A000120086049
:1008B000C6E71049002208310A608A06A2F85C00E7
:1008C00001200860BCE70B49002210310A604FF09C
:1008D0000052A2F8600001200860B1E7054900223B
:1008E00014310A604FF00052A2F862000120086043
:1008F000A6E700004009002210B55B4C00202060F4
:100900005A4800F09BFD0120206010BD10B54FF04B
:10091000E0214FF08060C1F88001C1F880025449A5
:10092000A02081F80004FFF7E7FF4FF00051C88CCA
:10093000CA8C00F00300120600EB400001D54D4ABE
:1009400001E04C4A303A12F8203001F8983F02EBAF
:10095000800042784A7082788A70C278CA700279C0
:100960000A7142794A7182798A71C279CA71027AAE
:100970000A72427A4A72827A8A72C07AC87210BD4A
:1009800070B54FF0005400F07F00049D84F88D0096
:1009900084F88E10A4F8942001213748002283B1F6
:1009A000C0F8801194F8913023F0700384F89130EE
:1009B00094F89130702606EA05152B4384F891309F
:1009C00001E0C0F8802114F8923F23F03403237033
:1009D000C0F84422C0F84012D0F89C110129FBD184
:1009E00070BDF0B54FF00054DDE90765DDE905C7DE
:1009F00000F07F0084F88D0084F88E10A4F8942015
:100A000084F88F30A4F896C001211B48002287B1DA
:100A1000C0F8801194F8913023F0700384F891307D
:100A200094F89130702707EA05152B4384F891302C
:100A300001E0C0F8802114F8923F23F034032370C2
:100A4000237843F02003237016B1C0F8481201E068
:100A5000C0F84822C0F84422C0F84012D0F89C11D7
:100A60000129FBD1F0BD000084140022AA820600F7
:100A70001AE000E0F0580000001000223748012181
:100A800001600021016070473548012101600021AB
:100A90000160704700B54FF0E0230122C3F88021C8
:100AA00003F5C073FFF7F0FFFFF7E8FF2C480838A5
:100AB0000260A02083F88002C3F8002143F8802C54
:100AC00000BD2749083910B1002008607047012097
:100AD000FBE723480121783801600021016070475D
:100AE00010B572B61F490C78002104E01D4A521C53
:100AF000525C4254491CA142F8DB40F6FC0000F075
:100B00009DFC62B6204610BD144901201C390860C6
:100B10007047144820300078124921310978401A72
:100B200000F03F0070474FF00051027881F800223A
:100B3000427881F80122827881F80222C27881F815
:100B40000322027981F80422427981F80522827910
:100B500081F80622C07981F8070270475C84002280
:100B6000940500220004002010B50A2000F05AF875
:100B70000B2000F057F80A2000F05FF80B2000F07F
:100B80005CF805210A2000F063F805210B2000F035
:100B90005FF84FF000507F2100F8351F4170C170A1
:100BA0000021C17101724172817210BD0123834025
:100BB000D8B24FF00053002993F8361001D001430A
:100BC00000E0814383F8361013F8381F0AB101435F
:100BD00000E081431970704701238340D8B24FF081
:100BE0000053002993F83C1006D0014383F83C10D1
:100BF00093F83E10014305E0814383F83C1093F8DD
:100C00003E10814383F83E1013F83D1F22B101438B
:100C100019709978014303E08143197099788143F1
:100C20009970704700F01F02012191404009800037
:100C300000F1E020C0F88011704700F01F02012190
:100C400091404009800000F1E020C0F88012704718
:100C50004907090E002806DA00F00F0000F1E02035
:100C600080F8141D704700F1E02080F800147047F0
:100C70007047FE4BFE4A998A814203D2401AD080C7
:100C8000084601E00021D180DA68FA491047F748A8
:100C900010B500698047F649C88810B1BDE810401A
:100CA000E7E78968002903D0BDE810400120084724
:100CB00010BDEE4810B500698047ED4C4FF00000C4
:100CC000A16819B188470020A06010BDFFF7D0FFD0
:100CD00010BDE749CA780B7952005A43E34B0878B4
:100CE000D2B29B6840F48070C96818470146182248
:100CF000DE4804F0D7BC38B5DD4A81791323117181
:100D00004179D170027901F0070102F01F028DF8DC
:100D100000208DF80110C078032200F01F008DF82C
:100D20000200D248694644681846A04738BDF8B565
:100D30000446007CCD4DC0F34002014662F35F01E2
:100D4000C0F3800241EA8201C0F3C00241EAC2015D
:100D5000C0F3001241EA0211C0F3401241EA42110D
:100D60008DF800108109607C272300F0010241EA20
:100D70000211C0F3400041EA40108DF80100607C90
:100D8000C0F38001C0F3C00241EA0211C0F30012B7
:100D900041EA4211C0F3401241EA8211800941EA5E
:100DA000C0108DF802006E68032269461846B047ED
:100DB000E0792B23C0F38002014662F39F01C0F368
:100DC000C10241EA0211C0F3401041EA80108DF8DF
:100DD0000000607CA17CC00901F0030140EA011021
:100DE0008DF801006E68022269461846B0472D262C
:100DF0002B680122694630469847A17C9DF8000087
:100E0000C1F3800108438DF800006B680122694638
:100E100030469847F8BD10B50446FFF76CFF2046F2
:100E200000F04FF92046BDE8104080E738B53D217D
:100E30008DF800108D49044612204B680122694646
:100E40009847A088FFF715FF38BD10B5044600F09D
:100E50007AF92046BDE81040E8E7F8B5834C122542
:100E60000646236801226946284698479DF80000F7
:100E7000012240F008008DF80000636869462846AA
:100E800098474825236801226946284698479DF8D7
:100E90000000012220F0060040EA46008DF8000024
:100EA00063686946284698472368012269462846B0
:100EB00098479DF80000012240F001008DF80000E5
:100EC0006368694628469847F8BD38B5674D482499
:100ED00001222B686946204698479DF800000122B0
:100EE00020F001008DF800006B68694620469847A5
:100EF00038BD38B55D4D2A2401222B68694620464D
:100F000098479DF80000012220F0100040F00100F9
:100F10008DF800006B6869462046984738BD38B5A3
:100F2000524D2A2401222B686946204698479DF895
:100F30000000012220F001008DF800006B68694676
:100F40002046984738BDF8B5484C442506462368E6
:100F500001226946284698479DF80000012240F08A
:100F600082008DF8000063686946284698472D2561
:100F7000236801226946284698479DF8000001220F
:100F800020F0FC0040F08E008DF800006368694698
:100F90002846984714252368012269462846984721
:100FA0009DF80000012220F0070040F001008DF8BC
:100FB0000000636869462846984715252368012282
:100FC0006946284698479DF8000006F01F0120F06A
:100FD0001F0001438DF8001063680122694628460E
:100FE0009847F8BD2DE9F843204C1325174688464D
:100FF00081462368012269462846984701269DF8C4
:10100000000006FA08F120F01F0001F01F01014363
:101010008DF80010636832466946284698472725B0
:10102000236801226946284698479DF80000BE4083
:1010300020F03F0006F03F0101438DF80010636887
:1010400001226946284698472E25236801226946D1
:10105000284698479DF80000012240F00C008DF8CA
:101060000000636869462846984705E018031000A9
:10107000380210003F0C00003E2023680122694620
:1010800098479DF8000000F0300189F80010BDE895
:10109000F883554B40F480701B681847524B40F45E
:1010A00080705B68184701B506209DF8001001228A
:1010B00001F01F018DF800104B494B6869469847B5
:1010C00008BDFEB5494D0446007828706078687008
:1010D000454EA078A870312733680122694638460A
:1010E0009847E07940069DF8000002D540F02000C6
:1010F00001E020F020008DF80000E179090602D51A
:1011000040F0800001E020F080008DF8000073685E
:10111000012269463846984721893220C1F30801E7
:10112000ADF80010E168CDF8021029788DF80610AE
:1011300069788DF80710A9788DF80810736809226E
:1011400069469847FEBD70B504460168274886B0D9
:10115000254D8160A168C160E1680161217C162094
:1011600001F001018DF80010617C8DF80110A17C67
:101170008DF8021000218DF80310A18A0F22C1F30F
:101180000C01ADF80410E18AC1F30B01ADF80610B3
:10119000218BC1F30B01ADF80810618BC1F30B017A
:1011A000ADF80A10A18BC1F30B01ADF80C10A17FB3
:1011B0008DF80E106B686946984731262B6801221E
:1011C00004A9304698479DF81000E17F20F01F00E9
:1011D00001F01F0101438DF810106B68012204A972
:1011E0003046984706B070BD180310003802100052
:1011F0004FF0E0214FF48030C1F88001C1F8800247
:101200007249A02081F80004704730B5704C012568
:101210002560E50603F03F0385F86B30002304E00A
:1012200051F8235040F823505B1C9342F8DB002018
:10123000206030BD30B595B00446302104F08EFA00
:101240006448006800906348001D00680190614890
:101250000830006802905F480C30006803905D48D9
:101260001030006804905B481430006805905948BD
:1012700018300068069057481C30006807905548A1
:101280002030006808905348243000680990514885
:10129000283000680A904F482C3000680B904D4869
:1012A000303000680C904B48343000680D9049484D
:1012B000383000680E9047483C3000680F90454831
:1012C0004030006810904348443000681190414815
:1012D0004830006812903F483F494C306FF002059B
:1012E00000681390009888424DD1A810A061206139
:1012F0002060A062E062E061206203A8029900F031
:101300006FF8019981423ED10B9845F2AA5180B203
:10131000884208D10498C0B2A061139A92B28A425E
:1013200000D0801DE0610C9880B2884217D10398EC
:10133000039A00F47F40D2B240EA0240039AC2F31B
:1013400007421043254A904203D30598C0F3012079
:1013500000E000202061059800F00F0020600D984B
:1013600080B2884201D10698A0620E9880B288426D
:1013700001D10798E0620F9880B2884201D10898A5
:10138000206215B030BDA56125612560A562E562CA
:10139000E5612562F5E710B50446142104F0DEF995
:1013A0000C487C38006820600A488038006860601B
:1013B000084878380068A060064874380068E06023
:1013C000044870380068206110BD000010E000E0A3
:1013D000441B0022B41E04005C000D6000010200EA
:1013E000F0B5074600200346184E10E057F823508A
:1013F00003224FEAC20C45FA0CF484EA2064E4B2FA
:10140000521E56F8244084EA0020F2D55B1C8B4221
:10141000ECDBF0BD70B5054600200C4C0246103CDC
:1014200009E0AB5C521C03F00F0604EB1313A65D3E
:101430001B78304418448A42F3DB70BD08B5009035
:10144000401E00900028FBDC08BD00003059000061
:101450004FF00051C88C4C4A00F0030012687AB17A
:1014600001280AD0022806D0032802D04FF41670B3
:101470000EE046200CE096200AE04FF4967007E05C
:1014800001280ED002280AD0032806D04FF4E170BC
:10149000401E21F8520F088070473220F8E76E2076
:1014A000F6E7DC20F4E748F61971480720F82A1F10
:1014B0000B2180F83E1000214183022180F8C010EA
:1014C0004FF008510120C1F8D4032F499839086022
:1014D0002E49086070474FF0005141F29840C8848F
:1014E000B6E74FF0005140F29A70C884B0E74FF071
:1014F0000050C08CA0F5A051983901D00020704751
:10150000012070474FF000518A8C60F304028A84F6
:1015100070471F48016841F00401016070471C4892
:10152000016821F00401016070474FF0005108810B
:101530007047174928310968016015491831096851
:10154000416013491C3109688160114920310968E3
:10155000C1600F492C31096801610D490C390968D6
:1015600041610B4914310968816170474FF00050A7
:10157000808870474FF00050807970474FF00051DD
:101580004C2081F820007047DC040022EC1B002274
:1015900010ED00E030B41DC8484981E81D0001216C
:1015A00030BC002003F062BE2DE9F84F444801240E
:1015B000006810F86C5F417890F846004D4300F0E9
:1015C000030004FA00FA3D486421103004F0C6F824
:1015D0003C4803F0EFF93B483B490471097809B9ED
:1015E00002210171DFF8D480002408F1100B36E0ED
:1015F000DFF8D090032735490026C9F80010484687
:1016000003F0DCF900226B460121104603F07EFE58
:101610000121002003F059FE98F8000060B102F0AB
:1016200094FB7F1E002F0AD0E9DC76B34FF0000058
:101630005946D8F804200FE04FF00106F5E74FF0C7
:10164000040003F0B0F9F0E751F8203032F91070DF
:101650003B4441F82030401CA842F5DB641C544553
:10166000C6DB012E11D1164900205C46184A0B68D2
:1016700009E093F8B26054F8201006F003063141F7
:1016800022F81010401CA842F3DB12490120087018
:10169000BDE8F88F10B50446002003F098FE022044
:1016A00003F095FEE00701D0FFF77EFF022003F074
:1016B000A9FEBDE81040002003F0A4BE30031000D6
:1016C000E00210004C021000050310004515000058
:1016D000523C01208C02100010B51C4C40F2FF114E
:1016E0002068FFF77DFE2168C1F8FC07FFF748F886
:1016F00000213F200EF1ACFAFFF742F82168BDE867
:1017000010403F234FF400721148FFF77EBD10B523
:1017100040F2FF310F48FFF763FE0E49C1F8FC0F9E
:10172000FFF72EF800213D200EF192FA00213E2015
:101730000EF18EFAFFF724F8BDE810403D234FF478
:10174000806204490448FFF760BD0000E002100019
:10175000F0EF03004C000120F0CF030030B41DC8AF
:101760004F4981E81D00012130BC002003F07EBDFF
:1017700010B5002003F02BFEFFF7BBFB00F064F870
:101780000446FFF7CCFB012C04D13C224549A020A4
:10179000FFF77FFC002003F035FE012010BD10B5DF
:1017A000FEF714FFBDE81040822002F0E1BA2DE9F7
:1017B000F047002003F00BFE00253B4F4FF0360AA8
:1017C0006E1EA846E8B2FFF76EFC0020FFF745FB4F
:1017D0003C683868A042FCD03868A042FCD133494C
:1017E0006420FEF7FBFEFEF79EFF81463868A042AC
:1017F000FCD03868A042FCD1FEF795FF0446FFF705
:1018000064FBFEF7E3FEA9EB040080B2B0EB0A0034
:1018100001D4014600E04142B14204D2002800DA7E
:1018200040420646A8466D1C6DB2202DCADB1D49FC
:1018300008F0FF00743981F8B000FFF734FCBDE810
:10184000F047002003F0DEBDFEB50025684603F03A
:10185000B1F8174800900320114E8DF8040004469B
:10186000684603F0ABF8002202AB0121104603F0FA
:101870004DFD0121002003F028FD307838B1641EB1
:1018800002F063FA002C05D0EADC2846FEBD4FF0DA
:101890000105FAE74FF0020003F085F8F5E70000D4
:1018A000A4031000C0000120981B00224F17000065
:1018B0000D17000030B41DC88E4981E81D000121BC
:1018C00030BC002003F0D2BC2DE9F84F8A480068F4
:1018D00010F86C4F40784443FEF75FFF8548642161
:1018E000103003F03BFF3221844803F015FF322112
:1018F000834803F011FF814842F21071323003F047
:101900000BFFDFF8F8A10020AAF1320A47F6FF71B9
:10191000AAF1320BCA4304E02AF810102BF8102069
:10192000401CA042F8DB774803F044F875490120D9
:1019300000250871DFF8CC9103267349DFF8B481E4
:101940000027C9F80010484603F038F800226B461B
:101950000121104603F0DAFC0121002003F0B5FC60
:1019600098F80000C0B102F0F0F9761E002E16D0F3
:10197000E9DCBFB36148D8F8041005FB04F200F1BC
:101980003200DFF8708100EB42034FF00000564652
:101990005F4608F1100823E04FF00107E9E74FF038
:1019A000040003F000F8E4E731F8102023F81020D9
:1019B00058F8202031F910C0624448F8202031F94D
:1019C000102037F910C0624501DD27F8102031F9E9
:1019D000102036F910C0624501DA26F81020401CAC
:1019E000A042E1DB6D1CC82DA4DBDFF808810020DC
:1019F000C821424D52465B4608F110080EE033F90B
:101A0000106032F91070F61B761025F8106058F847
:101A1000206096FBF1F648F82060401CA042EEDB07
:101A2000364F0020364E3237894615E0002258F8EE
:101A30002030114601FB040C37F91CC0BCEB030C31
:101A400001D5CCF1000C491C6244C829F2DB92FBA1
:101A5000F9F126F81010401CA042E7DB002707E050
:101A600036F9172035F91710F8B202F06DFB7F1C1C
:101A7000A742F5DBBDE8F84FFEF782BE2DE9F8433B
:101A800000248DF80040FEF788FE002003F09FFC44
:101A9000194D286890F86B00FFF755FA2F6800255C
:101AA000A1464FF00108A1370024785D08FA04F63A
:101AB0008DF8009006400DD0224629466846FFF773
:101AC00091FA9DF80000202804D1324629460520CD
:101AD00002F037FA641CE4B2062CE6D36D1CEDB2BA
:101AE000052DE1D3002003F08DFCFEF749FEBDE893
:101AF000F8830000B4031000E0021000B0100120D1
:101B0000F2370120540210006518000010B5044699
:101B10000221002003F0AAFB0F48046010BD08B5A5
:101B20000E48FEF74EFE00226B460221104603F0DF
:101B3000EDFB0221002003F0C8FB09485522016893
:101B400005480A7100684871020A8A71020CCA715C
:101B5000FEF7E7FC08BD00005C021000BD1A0000A3
:101B6000E402100008B50024DFF85881564F4FF406
:101B70000049264600226B464146104603F0C6FB4C
:101B80000098800319D5FEF741FC504804680660B0
:101B9000FEF73AFCE00701D0FFF709FEA00701D5E8
:101BA000FFF7E6FD00231A460121022002F0B3FAF6
:101BB0004FF40031002003F088FB0098000411D599
:101BC00000256D1CEDB2FFF7D3FD01286ED0032D6B
:101BD000F7D900224946082002F0B3F9494600200F
:101BE00003F073FB0098000510D5394804680660BF
:101BF0002046FFF74FFD4FF40061002003F065FB26
:101C00000023E1B21A46062002F085FA0098C004CB
:101C10000CD5FFF784FF002301221946022002F0B1
:101C20007AFA4FF48051002003F04FFB00988004B3
:101C300006D5FFF751FD4FF40051002003F045FB9E
:101C40000098400406D5FFF762FD4FF48041002064
:101C500003F03BFB0098400311D5386890F8A000D2
:101C6000C0070CD0FFF70AFF4FF48021002003F0DB
:101C70002CFB00231A4619460C2002F04CFA00985F
:101C800000037FF577AF386890F8A0008007F8D59B
:101C9000FFF71AFE4FF40021002003F016FB00238B
:101CA0001A4619460E2002F036FA63E70120FFF7C4
:101CB000F1FCE1B20023C4F30722082002F02BFA62
:101CC0008CE7000003F80F00E00210000003100092
:101CD000FC02100010B58143C80711D064480168A8
:101CE00041F0010101604FF40061002003F0BEFAF1
:101CF00001220023BDE810401146052002F00BBA76
:101D000010BDFEF7F2BC10B5FEF7EFFC0121BDE8F7
:101D10001040084603F0AABA5649012805D0022807
:101D200005D0032805D1042002E0022000E00320B2
:101D30000870704738B5002003F049FB4E48006832
:101D400010B1FFF7E9FF01E000F0CCF949484B4939
:101D50000078022813D003280ED0042812D00124C2
:101D60000025FEF7D6FE00B101256946032003F0E9
:101D7000BCFA009858B909E00868847AF0E7086866
:101D8000447AEDE70868B0F80B40E9E715B1142C88
:101D900000D2142420463A49FEF7AFFC0324394D03
:101DA00000F022FA012807D1287858B1641E01F00A
:101DB000CCFF002C0DD0F3DCBDE838404FF0000024
:101DC00003F020BB304801683048006800F01CF97F
:101DD000F2E7032002F0E7FDEEE770B52C48046857
:101DE0002C490D680C6095EA040F27D0214E2DB1C7
:101DF000A4B121462846BDE870406BE70220307050
:101E00001E4800680079000701D404203070214684
:101E10002846FFF75FFFBDE870408BE7FEF765FCE3
:101E20000121084603F051FA01203070214628466E
:101E3000FFF750FFBDE8704000F0F7B870BD10B577
:101E4000FEF753FC0121084603F03FFA094904203C
:101E5000087000F0B1F8BDE810406BE710B5FEF770
:101E600044FC0121084603F030FABDE8104061E768
:101E7000FC02100070021000F4021000E0021000DA
:101E8000B71C0000280410007C021000780210002B
:101E9000EC021000740210002DE9FC5F0E460028D1
:101EA0001BD055490978042917D1002A15D1DFF82C
:101EB0004C91DFF84C81534DD9F800109246097AC5
:101EC00049070ED5A978491CC9B2A970032906D8BB
:101ED000018808EB460020F8021CBDE8FC9F85F84D
:101EE00002A0032003F073FA454801906C78B5F91D
:101EF00004B02878274640B941480F235A46009439
:101F0000801D019902F074FB002734B93C4A5B46FE
:101F1000921D901D019902F05CFB39496F700C31E4
:101F2000B5F90420B5F90630002007E031F910407A
:101F30009C4201DD012404E0401CC0B29042F5DB6C
:101F40000024032003F05EFAD9F8000090F8E307BC
:101F5000DA2823D1D8F80010C8F81210B8F8041005
:101F6000A8F81610D8F80610C8F81810B8F80A1013
:101F7000A8F81C10D8F80C10C8F81E10B8F81010EB
:101F8000A8F822101E48C8F824A0C8F828A01230CB
:101F9000A8F82CA04682A9788182C4822C70002CDB
:101FA0009BD0FFF7AEFEBDE8FC5F0121084603F0C1
:101FB0005DB9144800787047124A012050700F48EC
:101FC0000068017A4B0790F8711002D590F86C30D8
:101FD00001E090F8703059439180B0F84B00D08008
:101FE0000021074811709170C1600182C0F806108D
:101FF000418100F0A9BADFE770021000E002100092
:10200000243801206002100070B5054630480C46A7
:10201000224690F90D102F484068FFF73DFF2146FA
:102020002846BDE8704000F014B810B5032003F056
:10203000CEF94821284803F091FB27490120087078
:10204000032003F0DFF90121BDE81040022003F076
:102050000DB92DE9F041DFF884800746002698F895
:1020600000000D4604282CD047EA0504032003F0A5
:10207000AEF9194A174B978115619868506098F826
:10208000000004281FD0FF2111751070E0070DD04B
:102090001348016811F86C0F49784843906042007A
:1020A0000D485968163003F0B8FA0126032003F0F2
:1020B000A9F9002E09D0BDE8F0410121022003F06A
:1020C000D5B80C46D2E7197BDEE7BDE8F081000009
:1020D00018051000280410005C05100070021000A4
:1020E000E00210002DE9F0417A4C0026DFF8E8818B
:1020F00020780227794D04280ED000F025FD012814
:1021000019D07748237802680320022B517B10D125
:1021100098F8003093B113E0FFF74BFF012803D08C
:1021200098F80000012804D16E49277001202E6024
:102130000870BDE8F08127702E60FAE7917B0420DB
:10214000127AD30701D19207F3D52A68521C2A606C
:102150008A42EEDD2E602070EBE730B41DC8624984
:1021600081E81D00082130BC012003F07FB82DE973
:10217000F0415B4800240068C17BC90732D05B494D
:10218000564E27460978C90727D0DFF84881012431
:1021900098F8001002290BD004290BD0857C00F0A0
:1021A000D3FC012808D05248007801280BD00EE05B
:1021B000457CF4E7C57CF2E798F80000042806D0D7
:1021C0000024776006E098F80000022807D07068C5
:1021D000401C70607068A84203DD776002E07760A1
:1021E000F8E700242046A4E72DE9FE4339483F4D97
:1021F000012600783F4FDFF80081032816D004281D
:10220000684610D0002402F0D5FBFFF7B0FF297814
:10221000C90700D0012440EA0401C90716D02E499D
:10222000097801B310E000F02EF812E068460024AF
:1022300002F0C0FBFFF79BFF2978C90700D00124FB
:1022400040EA0401C90701D08DF804603860C8F87D
:1022500000402A480090684602F0B0FB012806D0F2
:102260000020BDE8FE8302218DF80410EEE702ABEA
:1022700000220821012003F049F80821012003F081
:1022800024F80120EDE770B50446002502F092FB2A
:10229000FFF76DFF1249C3074FF0020205D009682E
:1022A000C97B89070FD504210BE0104B1B78DB0796
:1022B00000D00225AB0707D50968097A490702D57E
:1022C0000521217100E022710A4908600A48056071
:1022D00070BD0000700210000503100068021000BD
:1022E000E00210008C02100028041000740210009C
:1022F000E80210007C021000780210000B210000A0
:102300001C4808B500210122416002708160C16053
:10231000491E104602F0D9FFFFF76DFE6B46002202
:102320001721012002F0F2FF0098800705D5FFF782
:1023300054FD0221012002F0C8FF0098C00705D01B
:102340000121084602F0C1FFFFF7F4FC00984007A6
:1023500005D50421012002F0B8FFFFF770FD0098B9
:10236000C006DBD51021012002F0AFFFFFF776FD9C
:10237000D4E700007002100032216E4803F0CCB99F
:102380002DE9FC5F88466C4905466FF0130208682A
:102390004FF0010AC446037CB0F9167003F00F0435
:1023A000B0F91A30C4F11006B8F1280F15DB8B46CE
:1023B0004FF00009C18ACDE90019838A28223C2107
:1023C000604601F0F4FF07B2DBF800002822418BE1
:1023D000CDE90019038B3C2118E008F1140CBCF185
:1023E000140F17D84FF00109C18ACDE90019838A6B
:1023F00093460021404601F0DAFF07B24E48002123
:102400000068428BCDE90029038B5A46404601F013
:10241000CEFF03B24948DFF81CC1006881460AE0DC
:102420003CF9101035F9102001EB0708904515DB39
:10243000C91A914212DC401EF2D2BAF1000F0DD03F
:10244000494609E03CF9112035F91100624300FBCF
:10245000062000112CF81100491EF3D2BDE8FC9FA4
:1024600070B514460D46C00716D000F06DFB00286D
:1024700012D131480068C07B800703D5304800780E
:10248000042804D021462846BDE8704078E7284655
:10249000BDE8704000F001B870BD2DE9F04F26494D
:1024A000284C4FF0010E0A68DFF888B094F900401C
:1024B000117CB2F916A001F00F0692F86D10C6F16A
:1024C0001008B2F91A900B4614E093FBF1F7C3EB36
:1024D000440501FB1737EDB2FFB23BF9155030F957
:1024E000177005EB0A0CBC4522DBA5EB0905BD42C4
:1024F0001EDC5B1E012BE8DABEF1000F18D0DC46B3
:1025000014E092F86D50C1EB440391FBF5F705FB25
:102510001715EDB2DBB230F915703CF91350754365
:1025200007FB08552D112CF81350491E0129E8DA34
:10253000BDE8F08F523C0120E0021000A80210001C
:10254000A4021000A502100070B5FA4C002532213B
:10255000A4F807506572F84803F0DEF8F64A002048
:102560006FF00041503A42F82010401C1428FADB6A
:10257000F14A0020323247F6FF71CB4302F11406D4
:1025800022F8101026F81030401C0A28F8DB65707D
:102590002571E5706421E94803F0BEF8E74864213D
:1025A000643003F0B9F86571A57170BDF0B4E44C06
:1025B00000231A462478022C02D0F0BC184670473B
:1025C000E04B1C68E04B1E6874B900230AE030F948
:1025D000134096F8C950AC4201DCEC4201D501220F
:1025E00002E05B1C8B42F2D396F8B710F0BCD148E6
:1025F000093000F010BA2DE9F84F8246D248002683
:1026000047F6FF780468B346354694F8B100B4F84D
:10261000BA904307B4F8BC7094F8B8006FEA080C9D
:1026200005D5884222DC94F8B9308B421EDB884203
:1026300008DC94F8B900884204DBB4F8BF90B4F821
:10264000C17008E094F8C8004042884203DBB4F847
:10265000C390B4F8C570B849088810B100208E4600
:1026600013E032225146B44802F0D7FFBBE03AF9FA
:1026700010103EF810300E44C91A0BB2984500DD18
:1026800098469C4500DA9C46401C9042EFD3A949ED
:10269000A94A88783232009022F8108000981432CB
:1026A000A2F1960322F810C04A7800209E4643F813
:1026B0002260C0F114011144142391FBF3FC03FBCD
:1026C0001C180A315EF828C091FBF3F803FB1813BD
:1026D000401C5EF823100A28ACEB01010D44E8DB36
:1026E0009449C87810B1012804D007E04D4505DDB4
:1026F000012002E0FD4201D50220C8700A2095FBAE
:10270000F0F38E4D4879002725F81030401CC0B2F8
:102710004871322800D34F71C8788C46022844D1C2
:102720009CF80480B8F1280F3BD247F6FF73DFF81E
:102730000892D943002009F146097F4D323535F919
:1027400010509D4200DA2B4639F910508D4200DDC1
:102750002946401C0A28F0DBC81A784D9CF8061060
:102760006435634625F81100491CC9B28CF806107F
:10277000322900D39F7194F8BE1088420CDC1F717F
:102780004FF0010B8CF803700020714641F8206077
:10279000401C1428FADB08E008F101008CF8040062
:1027A00003E08CF804708CF8037000986546401CB8
:1027B000C0B28CF802000A2800D3AF70521CD0B20D
:1027C0006870142800D36F70322251465A4802F0C4
:1027D00024FFE97839B194F8E307DB2803D1142208
:1027E000552001F097FB5846BDE8F88F2DE9F04FD2
:1027F0008FB08346544A00200E9012688846BBF979
:10280000041092F8B520914250DDBBF906209142A8
:102810004CDD00244FEA58000D90DFF830914FF066
:10282000FF3A2746264625463421684602F096FFA1
:1028300042465946684601F09BFD434900206B46DD
:102840000A681BE033F91010B0EB580F08D292F869
:10285000B6C0614511DC761C2144F6B20CB20CE026
:1028600092F8B5C0614508DD6D1C0F44EDB23FB272
:10287000494502DD89460FFA80FA401C4045E1D304
:10288000BAF1030F0BD10D98864208D1854206D1CB
:10289000002C00DA6442BC4201DA01200E90254887
:1028A00092F8B71008300E9A00F0B5F80FB0BDE8F6
:1028B000F08F2DE9F05F8346994690468A460024C2
:1028C00002200A9E02F083FD1F4F1A4D3A6892F8CB
:1028D000B000C00720D0A4466146604608E038F941
:1028E000103092F8B340A34201DD491CC9B2401C2C
:1028F000B042F4D3B14201D14FF0010C0D4892F82F
:10290000B4106246C01D00F086F80446012801D0CC
:1029100014B130E0102032E0386890F8B000800741
:1029200018D531465046FFF761FF044601280FD005
:1029300084B120E080021000880410004E3801208D
:102940000503100098021000E00210000080FFFF55
:10295000112014E0386890F8B00040071AD53648C6
:102960000078B8B1324649465846FFF744FE04465F
:10297000012803D074B1012C02D005E01220287088
:102980000020A5F807006872022002F03BFD2046F7
:10299000BDE8F09F386890F8B0000007F4D572B237
:1029A00049465046FFF702FE04460128ECD11320A9
:1029B000E5E770B50646214D0C78002008702868C0
:1029C00090F8B100C00710D0022002F000FD1C48B2
:1029D0003146006842001B4802F01FFE1A480121E0
:1029E0000170022002F00EFD09E01848016841F074
:1029F000010101604FF40061002002F037FC2868FB
:102A00002246012190F8B100BDE8704000F00103BA
:102A1000052001F080BB10B500231C4642B10278AE
:102A2000521CD2B202708A4203D90470012300E022
:102A30000470184610BD000005031000E0021000ED
:102A4000A8021000523C01208C021000FC02100071
:102A500010B5F94C012019212070F84802F07EFED3
:102A6000F64832211A3002F057FEF44832214C3039
:102A700002F052FEF1490020083948602061E06010
:102A800060704FF4C8706061BDE810404FF49671FB
:102A9000EB4802F041BEF0B5EA48EB4C0122016878
:102AA0000020206060602081C4F80A00C4F80E0095
:102AB0006082E64801F13F0301F147060778E448E8
:102AC0000078384303D1E348007800B10222DFF8F0
:102AD00078C300200CF10A0C0EE033F81050554377
:102AE00024F8105033F8105016F800E0A5EB0E054E
:102AF00055432CF81050401C91F86C508542ECDC8A
:102B0000002F0AD0D4480078002806D1CB4831F8ED
:102B1000632F0838028089784180F0BDC948006879
:102B200090F8801069B1490010F88C2F521C407841
:102B30004A43C2EB022100F01F000141BE48C180A0
:102B400070470121F0E77047BB480069002800D0BA
:102B5000012070472DE9F04FB74C4FF0010A0AFAF7
:102B600001F5E468DFF8D4B22540BA4CABF1080BAC
:102B7000DDE909E72678B54C91464FF0000CBBF82B
:102B80000080247862460AD024B1BBF80220A8EB6A
:102B9000020292B2012F0AD04CB146B10BE00CB147
:102BA00006B142460FB904B12EB9A74A01E0A64AC0
:102BB0000A3232F81120A349096891F83A10CC077B
:102BC00030F919102ED0BEF1010F07D030F91340A3
:102BD0008C4200DC0C4694422BDC30E0002906DD00
:102BE00030F91340002C02DD0C4424B204E030F92B
:102BF00013408C4200DC0C4655EA07060BD0002D32
:102C0000E9D0002FE7D19142E5DA30F91300904284
:102C1000E1DA0024DFE79142DDDC30F91300904275
:102C2000D9DCF6E775B1914209DA30F91300904228
:102C300005DA0AFA09F00AFA03FC4CEA000C6046CD
:102C4000BDE8F08F9142F4DC30F913009042F0DCE3
:102C5000F5E72DE9F04115460024621E794E8EB04D
:102C60008046012941D13421684602F077FD7B4F2F
:102C7000414668463A6801F07BFB397840F6FF72BE
:102C800068462B6800F019FC6B49024628680B7BEC
:102C900020EA0303DB0708D03368B3F84F309342D0
:102CA00003DD20F001000124286083070BD50B7B96
:102CB0009B0708D43368B3F85530934203DA20F009
:102CC0000200A41C286043070FD5097B49070CD4D8
:102CD0003168B1F85730934203DCB1F85910914292
:102CE00003DA20F00400241D2860306890F8E30720
:102CF000DB2808D1002C06D00EB02146BDE8F041FB
:102D0000FD2001F007B90EB0BDE8F08101460020BA
:102D10008A0700D0012011F00C0F01D040F0020012
:102D200011F0300F01D040F00400704730B411783A
:102D300089073DD5B0F90430B0F906108B4237DD74
:102D4000002B00DA0023B0F90040002C00DA002448
:102D5000B0F90850002D00DA00252C44C4EB4303E1
:102D60001BB2002900DA0021B0F90240002C00DA81
:102D70000024B0F90A00002800DA00202044314C79
:102D8000C0EB410000B22168B1F84D10994201DC5E
:102D900081420DDD00211160216891F8E317DB29E4
:102DA00006D140EA0342012130BCFC2001F0B2B858
:102DB00030BC7047F0B50A680023002A1BD0214CB4
:102DC00003260022246894F85F50540024B230F99E
:102DD0001470AF4205DC00EB4404B4F90240AC428D
:102DE00001DD5B1CDBB2521C12B2B242EDDB032BE5
:102DF00001D100200860F0BDFCB50C460125CDE9ED
:102E000000540746052304220221FFF7A3FECDE963
:102E1000005406460022012311463846FFF79AFE69
:102E2000CDE9005406430323022201213846FFF76F
:102E300091FE3043C0B2FCBD8C021000203901204D
:102E400000EC0120E0021000E2041000043C01202C
:102E5000E80210000503100004031000A80210008F
:102E60002DE9F0410C4601463222FE4802F0D5FB26
:102E7000FC483222FC49323002F0CFFBF9483222C2
:102E8000FA49643002F0C9FBF849F648322232317F
:102E9000963002F0C2FBF54A0020FF23223A4FF0A1
:102EA000010E5668F24A0746EE49156814E00EFA1C
:102EB00000F2224201EB400C02D0ACF8C83001E035
:102EC000ACF8C870324201EB400202D0A2F8FA30EE
:102ED00001E0A2F8FA70401CA842E8D314E72DE9FB
:102EE000F843E44C8046E148894600252778257060
:102EF0003221963002F010FC17B1B8F8060020819C
:102F0000DD4EDB4C306890F82A10C9070AD00097D4
:102F100090F82B00414600F00F03208802B2D348FE
:102F200001F066FB022002F052FA2088CF4900B27D
:102F300000904B46CC4A01F1960001F095FA022030
:102F400002F060FAC94932229631A1F1320002F052
:102F500064FB3068C94FC07B000714D5C8480078AF
:102F6000012810D1387870B9C648007858B1208847
:102F7000BE4900B20090C448963102680846938E5C
:102F8000243201F056F92068B84942009631A1F187
:102F9000640002F042FBBD493878097808432FD11C
:102FA000306890F82A00400707D5B049227864318C
:102FB000012301F1320000F0ADFA306890F82A10D8
:102FC00089070BD590F86D100091A84990F86C30E6
:102FD00090F82C209631084600F01CFAA3493222C2
:102FE0009631A1F1320002F018FBA04A206832327B
:102FF00000904B4602F132014046FFF75AFC05466D
:103000002846BDE8F8832DE9F0410025984B064697
:103010002C46681E2A46AE46DFF858C21F680CE0F0
:1030200036F912308B4202DA0B44002B04DC012506
:1030300036F9124050B203E0521CBA42F0D3A5B1A7
:103040009CF80110491CC9B28CF8011032290ED924
:103050008F4A8CF801E001211160C3B2E2B2C4F3DF
:103060000721ED2001F057F801E08CF801E0284637
:103070004AE6814A10B5126804460020128C891A6B
:103080000BB27B49096806E034F911209A4201DC51
:10309000DA4200D50120491EF6D210BD70B5764D3A
:1030A000024600242868C07B40071CD51046FFF765
:1030B000E0FF012817D1FDF7A9F9764C206840F010
:1030C00002002060FDF7A0F94FF40041002002F05B
:1030D000CDF8286822780121C07BC0F38003072047
:1030E00001F019F80124204670BD30B56149624BEA
:1030F0000022CD681B68002D14464FEAC07505D02C
:103100007DB185070DD58D782DB10AE04DB18507CC
:1031100007D58C7005E001258D700C7193F89750E0
:10312000CD7010B18C7834B901E08C700C7102460E
:1031300093F89700C870104630BD10B54D4CA0787C
:10314000002805D0E07820B1401EE070207910B949
:1031500010BD01202071454803212238007901F07B
:1031600005FB0020A070207110BDF0B54A4C414F06
:103170000E4620780025A8B1B6F90600B7F9081068
:10318000081A00D540423C4900B20968B1F8601005
:10319000814207DA00204149207002200125087091
:1031A000FFF779FC38782178084301D1F08838811D
:1031B0002846F0BD2DE9F04704462C48DFF8B490CE
:1031C00022382A4F4568D9F81000002384EA000805
:1031D00029484FF0010A1A3F066820E00AFA03F076
:1031E00010EA080F10D0204220D023B1012B02D0CA
:1031F00096F83DC006E05FEA817C05D05FEAC47CBA
:1032000096F83BC007F803C017F903C0BCF1000FE4
:103210000FD0ACF1010C07F803C05B1C1BB293424A
:10322000DCDB2846C9F81040BDE8F08796F83EC0C0
:10323000E8E7204201D00543EFE78543EDE72DE9BC
:10324000F34F81B00B4D00240094B5F9061001989E
:10325000FFF7D9FE012843D0A846B5F9061001981A
:103260001EE0000000EC0120523C01203A39012010
:10327000A80210008C021000E0021000E80210000A
:10328000043C012005031000E4021000E9021000D4
:10329000F40210000003100006031000800210006A
:1032A000FFF7FCFE012829D0DDE90101FFF717FE39
:1032B000044601282ED002F00FFB01282AD0B54A7F
:1032C000DFF8D4A2B2481060DAF80010B34FB44E61
:1032D000C97B090725D5B349097801291CD020E00D
:1032E000B1480068012808D168694FF00051401EBC
:1032F000686111F8360F03D008700020BDE8FE8F1A
:1033000040F002000870887820F002008870A7481A
:103310000460FDE72046F1E7397811B99C4932395C
:1033200011603060002191461068FFF765FD0500CF
:1033300006D0387820B901213068FFF75DFD0540DF
:103340002846FFF7E3FC009004216846FEF762F888
:10335000974900F0FF0B38780978084323D1DAF851
:103360000000554690F83A00400704D56A46594691
:103370003068FFF76EFC0098A8B1286890F83A0012
:10338000800706D56A4659463068FFF7CFFC00989B
:1033900048B1286890F83A00000704D56946D9F882
:1033A0000000FFF707FD03224646D8F80C100098EE
:1033B000FFF700FF07460199FFF7D7FE744D863DE2
:1033C000A8B100246C602046029900F0D4FE287950
:1033D000214601F0CBF9012476480078042803D077
:1033E000DDE90010FFF73CFD6868F06092E768686F
:1033F00087420CD0F8B26F60FFF777FE0746287956
:10340000029900F0B8FE2879394601F0AFF9FFF7CC
:1034100094FEE1E72DE9FF4F9146864600250D9F7A
:1034200046E005FB07F00199012247F6FF7C01EB1E
:1034300040066FEA0C040EEB400B13460021C9F165
:10344000000A16E036F9110048450FDA50450DDD47
:10345000844500DD8446844200DA0446002802DA0E
:103460004FF0000202E001DD4FF0000301F1010125
:1034700089B2B942E6D352EA030009D012B1012A57
:1034800004D004E0012B02D1204601E023B100204A
:1034900041000BD0002107E06046F9E736F8112023
:1034A000121A2BF81120491CB942F7DB6D1CADB282
:1034B00003988542B5D3BDE8FF8F2DE9F041002484
:1034C000491E17468646CAB2A44626462546D80750
:1034D00001D002220DE098070BD50124032208E059
:1034E0003EF91400604502DD00FB04660544641CDF
:1034F000E4B29442F4D985FB012386FB070102F074
:1035000068F8002800DA0020791E884200DD0846AD
:1035100000B2E3E42DE9F04F00259B469AB0531E1C
:10352000DFB22C462B460DF1340AE94611E031F9A1
:10353000136035445E1CB44695FBF6F629F813601B
:10354000FE1A5B1C31F91680444494FBFCFC2AF8FB
:1035500016C09342EBDBBBF1010F01D1921ED2B238
:103560004C4655460FE034F9123035F912603344B9
:1035700003EBD3735B101BB2002B04DD31F8126038
:10358000F31A20F81230521EEDD21AB0BDE8F08FB7
:103590009E390120BC021000E0021000E802100079
:1035A000B8021000043C0120F40210005C09002263
:1035B000E902100070021000384808B50021C1600F
:1035C0008160416001210170354914200870FFF7C6
:1035D0003FFAFEF7D1FEFEF7B7FFFFF79FFA6B4603
:1035E00000220121022001F091FE0098C007F6D0D0
:1035F0000121022001F069FE00F001F8EFE770B54B
:103600000025032001F0E3FE00F024F8234C244EB3
:10361000207BC00705D096F900102069FFF70FFE48
:103620000546A06858B1022001F0D1FE96F90020AD
:103630002169A068FEF714FF022001F0E3FE012DCE
:1036400003D118492069FFF7B4F9BDE870400320A1
:1036500001F0D8BE70B5114C134DE068B5F90C10EF
:1036600080EA0102D20708D0C90702D0FFF7F0F9BB
:1036700003E0C00701D0FFF766FAB5F90C00E0607F
:103680002869A060A8686060074816302061287823
:103690002070287D60700548606170BDA402100034
:1036A000F8021000800210005C0510006C39012047
:1036B000094C00202060401C2060FDF76EF800F0EF
:1036C0004BFEFCF73DFF08B9FDF723FFFCF782FD39
:1036D00001F0B6FB2068EEE7C0021000E0490020D0
:1036E0000860E0490860E04908607047D0214DF665
:1036F000C062BA2000F025BC70B54FF40063984258
:1037000002D2DA4C246807E0A0F5805080B24FF472
:10371000805398420CD2D64C85189D4200DD1A1A6F
:10372000002303E0CD5C1E185B1CA5559342F9DB1A
:1037300070BDB0F5805F04D20A460146CB480068F0
:1037400008E0B0F5FE5F07D3A0F5FE5080B20A4650
:103750000146C74800F012BC704700F0A4BF10B586
:103760004FF40051002000F06EF90023BDE8104036
:103770001A461946032000F0CEBC10B54FF4804124
:10378000002000F060F90023BDE810401A461946F9
:10379000042000F0C0BCB2490A6882430A600221DA
:1037A000012000F050B9AE490A6802430A600221C4
:1037B000012000F048B9FDF78CB9FDF765B910B5E7
:1037C000C00711D0AB4800230222016841F001017B
:1037D00001600121052000F09EFCBDE810404FF47F
:1037E0000061002000F02FB910BD10B50324FCF7D4
:1037F0000DFEA1480460FCF707FE002301211A46D4
:10380000084600F088FCBDE810404FF4003100206D
:1038100000F019B910B5002301221946104600F036
:103820007AFCBDE810404FF48051002000F00BB945
:103830000421012000F007B98C4A904B012812683E
:1038400092F8E32709D002280CD0882A09D11978E8
:1038500000231A46172000F05EBC882AF7D00878AB
:1038600018707047882AFCD148781870EFE77E4AB4
:1038700000230128136005D1087810211060012071
:1038800000F0E1B870474FF48021002000F0DBB871
:103890004FF40021002000F0D6B8744800210068E1
:1038A00090F86800C00711D075480068827A12B19C
:1038B000FF2A03D00AE0C27A1AB107E0C27AFF2ACF
:1038C00004D196218172A521C172012100231A46DB
:1038D000102000F020BC6A4800210B4600680A4610
:1038E0008172C172202000F016BC10B50978654CB9
:1038F000002031B10121217063490870FFF7CBF836
:1039000000E020700120FFF75AFF00232178BDE876
:1039100010401A469A2000F0FEBB10B5594C227890
:10392000D2B9594A1278BAB1584A042809D00020AD
:103930001070002321781A469F20BDE8104000F047
:10394000EABB534B088818804888524908800120F8
:103950001070FFF7A0F8ECE7494A00EBD07013684D
:1039600020F0010203F1340001F057FE00231A4653
:1039700021789C20E1E7434A1278002A0BD00128E5
:1039800009DC3F480978002300681A4680F83A109D
:103990009D2000F0C0BB704770B53A4C2278A2B1B0
:1039A000374D00EBD07626F001022B6803F124009E
:1039B00001F033FE29687008002348842178BDE8AF
:1039C00070401A469B2000F0A6BB2F4800780028C4
:1039D00011D1264B304A314C1B6808E031F81050A9
:1039E00022F8105031F8105024F81050401C93F871
:1039F0006C508542F2DC70BD70B5214A4D78431E93
:103A000014680A781D445434202D02DBDBB2FF21F8
:103A100008E0A318421E1846491C01F0FEFD0023D1
:103A20001A460121BDE87040992000F074BB30B403
:103A30001B4C00B1087820700023C1B230BC1A467C
:103A4000A32000F068BB38B50C46054601F00EFC1B
:103A50006946284601F049FC009A2242F8D138BD57
:103A6000EC021000F0021000F4021000E00210005E
:103A70004C000120FC02100000031000F8021000AE
:103A8000E4021000E8021000043C012004031000CE
:103A9000183901201A390120E2041000EC0410004A
:103AA000E902100010B52021664801F035FE654896
:103AB000FDF716F86349401E11F8012BA2F190039F
:103AC0001F2B01D8604A05E0A2F1C0030F2B06D8D6
:103AD0005D4A803252F82320BDE810401047B82AD2
:103AE00021D00DDCB02A13D0B22A27D1032825D14A
:103AF00008888A78BDE8104040BA1146FFF719BE21
:103B0000FB2A17D0FC2A19D1BDE81040FFF735BEBB
:103B1000022813DD31F8022BBDE8104053BA821E93
:103B20001846FFF7E9BD022808D10888BDE8104013
:103B3000FFF713BEBDE81040FFF711BE10BD012016
:103B4000FFF731BE0120FFF726BE10B5FEF7FCFCE3
:103B5000BDE810400120FFF732BE00F057BA3B48E5
:103B600010B5017809B1022101703948394900685E
:103B700091F9003090F824219A420CDD90F81C0154
:103B800091F90010884206DAFEF7DEFCBDE810402D
:103B90000120FFF714BE10BD2C480178002903D086
:103BA00003210170FEF777BF704770B52A4D284C8E
:103BB0000020287020680078A52802D0012000F09D
:103BC000C9F840F2FF112068FDF70AFC2168D1F81E
:103BD000FC17814202D0022000F0BCF840F2FF3115
:103BE0001E48FDF7FDFB1D49D1F8FC1F814206D0A0
:103BF00020680079800702D4032000F0ABF8184851
:103C0000007881074FF0010001D5287070BD0F4981
:103C10000870FEF740FFBDE870400120FFF7CFBD00
:103C20000A4910B500200870FEF735FF0848006803
:103C3000007A800701D5FFF7FBFDBDE810400120A9
:103C4000FFF7BDBDF6041000305D00000503100055
:103C5000E0021000F8021000060310004C000120E2
:103C60001C39012008B5FFF739FD00F0B2F91B4CF3
:103C700020680079800701D5FFF7B7FD206800793B
:103C8000C00701D0FFF75BFF2168C87B00070DD597
:103C900011F86C0F4978484300F096FA1049002358
:103CA0001A4608700146C02000F035FAFEF7F3FE10
:103CB00001216B460022032001F028FB0098C00779
:103CC000F6D0FFF7EFFE0121032001F0FEFAFCF72A
:103CD0001BFFEDE70121032001F0C8BAE00210004C
:103CE000043C0120304C2F4AC4E900210168A16046
:103CF0004168E16081682161C16861610169A16118
:103D00004169E16181692162C069606204F1280052
:103D1000FDF70FFC01F013FC606400F035F8224958
:103D2000224AC1E90020704710B501284FF0000277
:103D300005D00146BDE81040022000F002B9012183
:103D4000022000F0FEF800F01FF8012801D1022047
:103D5000EAE7704710B5044601460022032000F050
:103D6000F0F8012C01D0022C01D100F00DF810BDAB
:103D700000220146062000F0E4B801460022072098
:103D800000F0DFF800F000F8FCF707FD4FF00050FE
:103D900010F8361F41F002010170817821F0020114
:103DA0008170FEE7AF0550FA00EE0120BA0110ABBA
:103DB00077B585B00E46BDF814401546200A40EA96
:103DC0000420ADF814004F48BDF814100024018001
:103DD000A0F58070CDE900044B480294039400687C
:103DE0001346484AC0790221FCF7FBFD08B02A4679
:103DF0003046BDE87040454901F00FBC17B581B0B1
:103E00000B46BDF804001446010A41EA0020ADF853
:103E100004003C48BDF8041020F8021B194601F0CC
:103E2000FCFB0020009038480023364A0068A11CA3
:103E3000C079FCF7A5FD1FBD77B585B00E46BDF86E
:103E400014401546200A40EA0420ADF814002D481D
:103E5000BDF81410002401802C48CDE900042A4844
:103E60000294039400681346264AC0790221FCF7A5
:103E7000B8FD08B02A463046BDE87040234901F03D
:103E8000CCBBFCF76DBB08B50020ADF800000222EA
:103E90006946FFF78DFFBDF8000008BD00B587B08B
:103EA000002201210720FCF781FE072001F002FD1E
:103EB00000204FF4FA7100BF401C8842FBDB072052
:103EC00001F001FDFFF7DFFFA0F584410E3902D0BC
:103ED0000120FFF729FFAFF2DB000190AFF22F10B6
:103EE0000090AFF2AB000290AFF269000390084877
:103EF000049040F28F20ADF814006846FCF7F6FEFF
:103F000007B000BD043B0120E0021000043A01208C
:103F1000030500001CB5DB238DF800308DF801008F
:103F20008DF80210100E8DF80300100C8DF80400AF
:103F3000100A8DF805008DF80620684600F032F969
:103F40001CBD1CB50F238DF800308DF801008DF8D5
:103F50000210080A8DF803008DF80420100A8DF86D
:103F60000500100C8DF80600100E95498DF807001D
:103F7000012008706846FCF7D6FD1CBD2DE9FC4108
:103F8000002706460097122015460C4601978DF82B
:103F900000001AE0200A8DF80100C4F30B008DF830
:103FA0000240315C30448DF8031041788DF80410E4
:103FB00081788DF80510C0788DF806008DF80770AF
:103FC000684600F0EFF8241D2D1F002DE2DCBDE84F
:103FD000FC811CB500207B490090019009681023EA
:103FE0004A7889788DF800308DF804008DF801004A
:103FF0008DF805208DF802008DF806108DF803006D
:104000008DF80700684600F0CDF81CBD70B588B08B
:1040100000240094142001948DF80000FDF7AAFA02
:104020008DF8010022208DF80300664E65208DF882
:1040300004003068624D41788DF8051080788DF865
:104040000600287880018DF80700684600F0AAF87D
:104050000094152001948DF80000306890F8EC175A
:104060008DF8011090F8ED178DF8021090F8EE170A
:104070008DF8031090F8EF078DF804002878800180
:104080008DF80700684600F08DF8009402A80194AE
:10409000FDF781F91B208DF800000298000E8DF8C5
:1040A00001000298000C8DF802000298000A8DF8B9
:1040B000030002988DF804008DF8054004988DF8EF
:1040C0000600287880018DF80700684600F06AF83D
:1040D00000941C208DF8000003980194000E8DF8C8
:1040E00001000398000C8DF802000398000A8DF877
:1040F000030003988DF8040005988DF805000698D4
:104100008DF80600287880018DF80700684600F0D9
:1041100049F808B070BD1CB52A4C246894F8E247F1
:10412000A40710D500240194009416248DF80040B3
:104130008DF801008DF802108DF803208DF8043001
:10414000684600F02FF81CBD1CB5002300930193B6
:10415000E1238DF800308DF80100080A8DF8020087
:10416000100A8DF804008DF803108DF805206846BC
:1041700000F018F81CBD1CB5124A126892F8932082
:10418000D2070ED0002200920E2301928DF800304B
:104190008DF801008DF806108DF80720684600F0B4
:1041A00001F81CBD10B50446012001F010F92046AD
:1041B000FCF7B9FCBDE81040012001F023B9000074
:1041C000C4021000E0021000F0B5234907460120A8
:1041D0000A68518C59B32149096891F8693092F8FD
:1041E0003A108B4202D009B1FF2920D102F13406E6
:1041F00002F12404B51C00214FF6FF7C383208E0A0
:1042000034F811300BB1634501D1002003E0491CA3
:1042100089B2B942F4D3318809B1FF2900D1002015
:10422000298821B1FF2902D01288914200D20020B2
:10423000F0BDF0B50024059E0AE031F9145032F8C3
:1042400014705D4395FBF7F520F81450641CA4B27C
:10425000B442F2DBF0BD0000E4021000E002100006
:1042600070B54A21304801F057FA2F4CA6202F4D47
:10427000208042F265206080286841782171807832
:104280006071FDF773F9E080FFF7FDFD208128687C
:1042900090F86C10217790F86D1061772449E183D4
:1042A00024492184244961842449A1872449A18483
:1042B0002449E18424492185D0F8FC170A0C628541
:1042C000A185B0F83F10E185B0F841102186B0F823
:1042D00043106186B0F84510A18690F8741001F083
:1042E000030284F83620C1F3011184F8371090F8E6
:1042F000681001F001012187144909684A8952BAFE
:10430000628701F12202E2873232A4F8422090F85B
:10431000690004F8440F91F83A0060700C4824F8E2
:10432000020F0C48608070BD00000120E002100008
:10433000063C01203A3901206C3901209E390120C8
:10434000523C0120C00001201C390120E402100071
:10435000183901201A39012010B5FCF757F8FDF77C
:10436000C6F808B1FDF7BDF8BDE81040FCF74CB841
:1043700030B501230CE000EB430531F8134025F87C
:10438000024C01EB430434F8024C20F813409B1C10
:104390009342F0D330BD10B5FCF738F8FDF7A7F81D
:1043A00008B9FDF798F8BDE81040FCF72DB8F0B556
:1043B000851ADDE905471E1B75438E1A012F02D0B1
:1043C000904206DD0BE0904201DC1846F0BD8842C9
:1043D00001DB2046F0BD95FBF6F0181AF0BD8842CF
:1043E000F3DA95FBF6F02044F0BD2DE9FC4F0446CE
:1043F0008F480B4600260768354607F58A7207F591
:104400008E7C125707F5927807F5967107F59A7921
:1044100007F59E7A07F5A27B184607F5A6779A421C
:1044200000DD10460957994200DA084682420ADC4C
:104430001CF90430834206DB194619F904300125C2
:104440001AF9044008E018F90420824209DC81428C
:1044500007DB3B571BF90440CDE90045FFF7A7FFF9
:1044600046B23046BDE8FC8F2DE9F84F89467049C9
:104470000546DFF8C0A108689B46904690F8E30720
:10448000882808D12A68CAF800206A68CAF8042077
:10449000AA68CAF8082000245AE0674839F81410BE
:1044A000634B076838F814000126081A25F8140031
:1044B0001868243790F8E317882906D139F81420B2
:1044C00038F81410511A2AF81410C07BC0063DD5D4
:1044D0005A480078D0BB5A480078012836D159484C
:1044E000007898B3A0B25946FFF77FFF01465048C5
:1044F000006890F8E307882805D1534880F830B267
:10450000204480F831120AEB44008181F1B135F981
:10451000140064225043C1F1640290FBF2F000B237
:10452000002802DA0026404200B237F81420824206
:1045300005DC821A4A43642192FBF1F1401A25F806
:1045400014001EB980B2404225F81400641C24B245
:104550000A988442A1DB3648006890F8E30788286F
:1045600035D12968CAF818106968CAF81C10A968FA
:10457000CAF82010062000902F482E4902681831F2
:1045800001F10C00938E2432FFF753FE2E4F2F4E75
:104590006FF0130530883D54401C30800024A0B2D9
:1045A0002946FFF722FF3188641C24B27854491C45
:1045B0003180062CF3DB6D1C6DB23C2DEADB3088BC
:1045C000B0F50C7F07F800B001D300203080BDE8C3
:1045D000F88F70B5002408E031F8145032F81460F8
:1045E000AD1B20F81450641C24B29C42F4DB70BD57
:1045F000F0B4049C012C04D01BB1C3F110060024BC
:1046000012E0F0BC520001F008B830F9145031F952
:1046100014705D4307FB0655EF1705EB17752D1159
:1046200020F81450641C24B29442EEDBF0BC7047B6
:10463000E0021000BC3E0120E4021000E80210007D
:10464000043C012005031000843C0120C602100038
:104650000FB42DE9F05F0025DDF874A08B4681468C
:104660002E464FF0010808FA06F7002407EA0B0768
:104670006FB108FA04F010EA090F08D0324621465B
:104680000C9800F0CFFA0AF805006D1CEDB2641C1E
:10469000E4B2052CECD3761CF6B2052EE3D3BDE8CC
:1046A000F01F5DF814FB10B5044650212B4801F0B3
:1046B00033F82B4A1178491C1170A00504D5BDE8C8
:1046C0001040264800F001B810BD2DE9F041044625
:1046D00090B0A52020704FF40070A4F8010000F005
:1046E000A8F9207100F0A0F9607100F098F98046F7
:1046F00000F090F905461B4800680179552904D15E
:10470000D0F8050020F07F40A060174E392206F156
:10471000740796F8B000207304F130000F90391D33
:10472000684600F0BFFF002229464046736FFFF73E
:104730008FFF04F110000F903922391D684600F0F8
:10474000B1FF012229464046736FFFF781FF0448FD
:104750000078E07010B0BDE8F0810000008001201A
:10476000C8021000E40210004C00012070B5854E14
:1047700005460C46306890F8940001070AD5E10719
:1047800000F007004FF0000201D0012100E00021FD
:10479000FCF70CFA306890F8941008060AD5A007C8
:1047A000C1F302104FF0000201D5012100E0002109
:1047B000FCF7FCF9306890F8950001070AD5690705
:1047C00000F007004FF0000201D5012100E00021B8
:1047D000FCF7ECF9306890F89610080712D56A4893
:1047E000007878B16948007860B96948007848B9BC
:1047F0006848007800284FEA847008D0002810D15B
:10480000A8070ED101F007000022114605E000289C
:10481000F6D001F0070000220121BDE87040FCF74E
:10482000C5B970BD10B5574C206890F894000107C9
:104830001CD500F0070001F046F8206890F89400BD
:1048400000F0070001F036F820680022114690F8C9
:10485000940000F00700FCF7A9F920680022114637
:1048600090F8940000F00700FCF7B6F9206890F883
:10487000940001061CD5C0F3021001F024F8206852
:1048800090F89400C0F3021001F014F820680022A0
:10489000114690F89400C0F30210FCF787F92068E5
:1048A0000022114690F89400C0F30210FCF794F92E
:1048B000206890F8950001071CD500F0070001F072
:1048C00002F8206890F8950000F0070000F0F2FF71
:1048D00020680022114690F8950000F00700FCF7D0
:1048E00065F920680022114690F8950000F0070055
:1048F000FCF772F9206890F8950001061CD5C0F30A
:10490000021000F0E0FF206890F89500C0F302105C
:1049100000F0D0FF20680022114690F89500C0F307
:104920000210FCF743F920680022114690F8950028
:10493000C0F30210FCF750F9206890F896000107C8
:104940001ED500F0070000F0BEFF206890F896002A
:1049500000F0070000F0AEFF20680022114690F83A
:10496000960000F00700FCF721F9206800221146AC
:1049700090F89600BDE8104000F00700FCF72CB955
:1049800010BD0000E002100005031000E802100056
:10499000E90210009002100010B500F001F91B4967
:1049A0000020086010BD10B5FFF7B9F9BDE8104050
:1049B000FCF78FB8002101604160704710B50179A4
:1049C00099B1134900220A604A608A60CA600F499F
:1049D000D0E90020C1E90120081D00F01FF90B48B3
:1049E000001D00F0B3F9012010BD002010BD10B56E
:1049F0000749064C087020688860201D016804483B
:104A000088472068401C206010BD0000CC021000C8
:104A100018051000FD48006890F86A007047FB48D0
:104A2000006890F86B007047F848006890F86C00D8
:104A30007047F648006890F86D00704770B5040044
:104A400004D1FCF746F9F349F1484860F248F34ACB
:104A5000002101701160F24801230360450685F8CA
:104A6000EE10F04EA0253560016013602046BDE8D1
:104A70007040FFF7BCBF10B50446142100F06EFE75
:104A80000020207080206070A020A070FFF7C7FF7A
:104A9000E070FFF7BFFF2071FFF7C6FF6071FFF7FF
:104AA000C8FFA071D948E279006810F8771F61F358
:104AB0008612E27110F80519490861F3C712E27114
:104AC000C18821818168E1600378217C63F3000162
:104AD000217403785B0863F34101217403789B0818
:104AE00063F3820121740378DB0863F3C30121744B
:104AF00003781B0963F30411217403785B0963F3E2
:104B00004511217403789B0963F38711217443785D
:104B1000617C63F30001617443785B0863F34101D6
:104B2000617443789B0863F3820161744378DB0806
:104B300063F3C301617443781B0963F30411617467
:104B400043785B0963F34511617443789B0963F310
:104B500086116174837863F30102E27183789B08A4
:104B600063F38202E27183781B0963F3C402E2718A
:104B700083789B0963F34512E271C27862F3C7112F
:104B80006174C1780A09A17C62F30101A174007902
:104B900060F38201A1742046BDE81040FCF73BB9E8
:104BA0002DE9F0419C4800244FF0E0270470447048
:104BB0008470C47004714FF080764FF00108C7F81C
:104BC00080619948A02580F8005420229749984890
:104BD000843700F067FD9348083805609548046005
:104BE0008F49091DC1F80080710181F8DE80C7F886
:104BF000FC61FE673D229049A020FCF74FFA8E48E9
:104C0000743890F8B000FCF74EFA8C48FFF733FF89
:104C1000BDE8F0418948143000F0D4B87E49002046
:104C200008707047844B02EB4202743B03EB820234
:104C300002EB410110B191F87500704791F87400D2
:104C400070472DE9F041DFF8C4C102460024714DE0
:104C50000127714BDCF80000052912D0042949D046
:104C6000FFF7DDFED070FFF7D5FE1071FFF7DCFE19
:104C70005071FFF7DEFE9071BDE8F0411046FCF781
:104C80003AB8017A490726D593F903100CE090F859
:104C90006E6007FA01FE16EA0E0F04D0D97019797A
:104CA000491C197102E0491C0529F0DBD97890F8FC
:104CB0006A6007FA01FE06EA0E061671577193F94B
:104CC00004606E73491CD97090F86C10B14209DC15
:104CD000DC701C7106E06C7390F86E10117190F826
:104CE0007010517190F86F00D070DCF8000090F8EF
:104CF0007100C0E793F901100CE090F86A6007FAC0
:104D000001FE16EA0E0F04D059709978491C99706B
:104D100002E0491C0529F0DB5771597810F86A6FD9
:104D20008F403E4016714078D070DCF80000491C7E
:104D300090F86D60967193F902602E73597090F837
:104D40006C00B04298DC5C709C7095E730B50479DB
:104D500089B0B4B12021684600F000FD6D462146BF
:104D60003648FFF76EFF354920221431284600F0FF
:104D700099FC0025062C10D2DFE804F00F0F060D79
:104D8000060609B0012030BD2048006890F8900068
:104D90008DF8110001E08DF81F506846FCF755F8BA
:104DA0001D49012008701F480C380560112041077B
:104DB00081F8EE00E5E718480078012801D1FBF7FB
:104DC00078BF7047AFF28B31016011498160323199
:104DD000C160002101740D49096811F8802F4274E7
:104DE0004A7882744A8882828A88C282CA88028308
:104DF0000A8942834A8982830A7B8277497B01F050
:104E00001F01C17741F2883181807047E0021000B4
:104E1000063C012018051000D802100010050022E1
:104E2000901B0022100C022018E000E0F05D000052
:104E300000000220E01E0022C00001202805100012
:104E400010B5FCF76CFBFBF79BFCBDE81040FFF7CF
:104E5000A2BA0AF11FBF10B5FFF7F2FF10BD10B5DF
:104E6000FFF7EEFF10BD10B5FFF7EAFF10BD10B55C
:104E7000FFF7E6FFBDE81040FEF72CBF10B5FFF7C7
:104E8000DFFF10BD10B5FFF7DBFFBDE81040FBF7FB
:104E90007DBB10B5FFF7D4FFBDE81040FBF7B4BBF6
:104EA00010B5FFF7CDFFBDE81040FBF7D6BB10B53E
:104EB000FFF7C6FF10BD10B5FFF7C2FFBDE81040F9
:104EC000FBF7F3BB10B5FFF7BBFFBDE81040FBF7E6
:104ED00032BC10B5FFF7B4FF10BD10B5FFF7B0FF3F
:104EE00010BD10B5FFF7ACFF10BD10B5FFF7A8FF60
:104EF00010BD10B5FFF7A4FF10BD10B5FFF7A0FF60
:104F000010BD10B5FFF79CFF10BD10B5FFF798FF5F
:104F100010BD7047704710B5FFF792FFBDE8104015
:104F2000FBF76BBC704770477047704710B5FFF7D1
:104F300087FFBDE81040FFF73EBF704730B58DB02A
:104F400042F26520FCF7F1FAFCF7ADFA4FF400628B
:104F50004B494C4800F0A6FB4FF480524A494B485D
:104F600000F0A0FBFBF796FD0120FBF7AAFDFCF784
:104F70003FF90E246846FCF75DF90698C01C65D021
:104F80000698401C64D00698801C61D00698C4B274
:104F90002046FCF7B7FAFCF79EFAFCF7EFFA3C4C18
:104FA00020680078A52802D00120FEF7D3FE40F249
:104FB000FF112068FCF714FA2168D1F8FC17814230
:104FC00002D00220FEF7C6FE40F2FF312F48FCF768
:104FD00007FA2E49D1F8FC1F814206D020680079DB
:104FE000800702D40320FEF7B5FEFBF7BDFDFBF7FB
:104FF0000FFA2948274D0168087955282CD07020D0
:10500000FEF7B6FE2846FBF78CFAFBF77FFC20681C
:105010000079400704D4214900200860091F086076
:10502000FEF73CFFFFF7B8FCFBF7BCFB38B10022F2
:1050300011460120FEF785FF0120FEF770FEFBF709
:105040009AFB0DB0BDE83040FFF7ECBB312000E02B
:105050003020FEF78DFE9BE7D1F8050020F07F455C
:10506000D0E710B5FBF7D2F9FFF768FFFFF7F8F8C4
:1050700000F016F8FBF7C8F900F07EF8012010BD2B
:10508000F0EF030000F00120F0CF03004C000120FE
:10509000E002100000770100E402100084140022F6
:1050A0007FB500F041F81F4D002405EB441000F1DE
:1050B0001002017F4CCACDE90261CDE900230FC87F
:1050C00000F0DAF910B10220FEF757FE641C052C3F
:1050D000EBDB144D0024A03504EB440005EB80010C
:1050E00055F820008A68496800F046F910B102209E
:1050F000FEF743FE641C042CEEDB0A4D0024D03581
:1051000005EBC400416855F8340000F08FF810B189
:105110000220FEF732FE641C042CF1DB7FBD03206D
:10512000FEF72BBE105E00001A4910B50120087072
:10513000194900200860194908601949086019498F
:10514000086000F07DF900F00FF900F067F800202A
:1051500010BD10B5124800F024FA104908600E493D
:105160000968884207D00B480078022803D1BDE8BF
:105170001040FBF703B910BD10B5FFF7EAFF054972
:1051800002200870FBF7DEF84FF0FF3010BD05205D
:105190007047000007031000080310000C03100004
:1051A000100310001403100070B50D460446C169C9
:1051B0008068CC2200F0A8FAE169A0680844403871
:1051C0004FF08071C163216A8163002141630163F3
:1051D000C1628162C0E908514FF00B31C1614FF0EB
:1051E0000A3181614FF0093141614FF008310161AD
:1051F0004FF00731C1604FF0063181604FF005314B
:1052000041604FF00431016070BD82698168914254
:1052100002D84068FFF783BF7047000010B54FF415
:10522000B4714F4800F09AFA002010BD70B50546E1
:1052300000EBC5014A4800EB8104FBF7D7F80646AE
:10524000207828B13046FBF7D9F86FF0010070BD27
:105250000320207000206560206204F11C0000F033
:1052600079F93046FBF7CAF8002070BD2DE9F0410E
:105270000F463B49002500EBC00001EB80042E46A1
:10528000FBF7B4F88046206A3843206204F11C0022
:10529000074600F086F90CE0216A026C114203D047
:1052A00000F026F9012600E06D1C2946384600F082
:1052B0006EF90028F0D1012E01D1FFF74AFF4046D8
:1052C000FBF79CF80020BDE8F08170B50D4624493D
:1052D00000EBC00001EB8004FBF788F8216AA943CA
:1052E0002162FBF78BF8002070BD70B50C461C499D
:1052F00000EBC00001EB800500202060FBF776F892
:10530000296A2160FBF77AF8002070BD2DE9F04191
:105310000D46134900EBC0001E46904601EB800489
:10532000FBF764F807460F4800680564216A2942C4
:1053300003D104F11C0100F0EDF83846FBF75EF8EC
:10534000FBF754F8216A29403160B8F1010F02D10E
:10535000216AA9432162FBF751F80020B3E700005E
:10536000641910000803100010B54FF4C8713248DA
:1053700000F0F4F9002010BD2DE9F0418846054603
:105380002D4900EB8500174601EBC004FBF72EF812
:105390000646207830B13046FBF730F86FF0010058
:1053A000BDE8F08102202070E7611422414604F13B
:1053B0000800656000F031F90020206204F124004B
:1053C00000F0C8F83046FBF719F80020E8E770B5A0
:1053D000194900EB800001EBC004FBF707F8054614
:1053E000D4E90701814205DB144804F12401006877
:1053F00000F090F8206A401C20622846FAF7FEFF71
:10540000002070BD70B50C4900EB800001EBC004BA
:10541000FAF7ECFF0546206A08B1401E206204F14D
:10542000240000F0BEF810B1606A00F011F82846C0
:10543000FAF7E4FF002070BDCC1A1000080310003A
:1054400010B54FF42A71404800F088F9002010BDD3
:1054500010B5044690F8380002280BD0204600F022
:10546000A2F8022084F838003849204600F076F887
:10547000FFF76FFE002010BD2DE9F05F8B4606465A
:10548000314900EB06109046DDE90AA911F8202009
:105490001D461AB16FF00100BDE8F09F01EB8004DA
:1054A000FAF7A4FF074601202070C4E90165C4E9AA
:1054B0000585C4E907A91422594604F1240000F027
:1054C000ACF8002084F8370084F838006169E060A7
:1054D0002061C4E90F1020460C99FFF765FEA0601B
:1054E0002046FFF7B5FF3846FAF788FF0020D3E7DC
:1054F00010B5044690F83800022809D0204600F084
:1055000052F8022084F838001049204600F026F8AE
:10551000002010BD70B5044690F838000D460228F2
:105520000BD1204600F03FF8032084F838002946CC
:10553000204600F013F8FFF70CFE002070BD044871
:1055400000684068704700005C1C100010031000E9
:1055500008031000002101600846704730B50A6852
:1055600012B10B46C46B09E000220860C0E90321B8
:105570000BE000BF02F10C03D26812B1D56BA5425B
:10558000F8DC1A68C0E903211860002030BD00680B
:10559000002201E0C068521C8A4201D00028F9D1E3
:1055A00070470068704702690AB1116831B96FF03D
:1055B0000400704701F10C02C96839B18142F9D188
:1055C000C968116000210161084670476FF003004F
:1055D000704710B54C1084EA530404D54042C1F121
:1055E000000138BF491E1B4204D55242C3F10003DB
:1055F00038BF5B1E00F0D9F814F0804F04D0404251
:10560000C1F1000138BF491E14F0004F04D05242CE
:10561000C3F1000338BF5B1E10BD032A40F2308087
:1056200010F0030C00F0158011F8013BBCF1020FE3
:10563000624498BF11F801CB00F8013B38BF11F864
:10564000013BA2F1040298BF00F801CB38BF00F87B
:10565000013B11F0030300F02580083AC0F00880F8
:1056600051F8043B083A51F804CBA0E80810F5E7DC
:10567000121D5CBF51F8043B40F8043BAFF30080BF
:10568000D20724BF11F8013B11F801CB48BF11F834
:10569000012B24BF00F8013B00F801CB48BF00F804
:1056A000012B704710B5203AC0F00B80B1E81850BC
:1056B000203AA0E81850B1E81850A0E81850BFF4FC
:1056C000F5AF5FEA027C24BFB1E81850A0E818509B
:1056D00044BF18C918C0BDE810405FEA827C24BFEF
:1056E00051F8043B40F8043B08BF7047D20728BF7D
:1056F00031F8023B48BF11F8012B28BF20F8023BCC
:1057000048BF00F8012B704702F0FF0343EA032271
:1057100042EA024200F002B84FF000020429C0F051
:10572000128010F0030C00F01B80CCF1040CBCF1D3
:10573000020F18BF00F8012BA8BF20F8022BA1EB25
:105740000C0100F00DB85FEAC17C24BF00F8012B0A
:1057500000F8012B48BF00F8012B70474FF0000202
:1057600000B5134694469646203922BFA0E80C5057
:10577000A0E80C50B1F12001BFF4F7AF090728BF32
:10578000A0E80C5048BF0CC05DF804EB890028BFAE
:1057900040F8042B08BF704748BF20F8022B11F0D7
:1057A000804F18BF00F8012B704753EA020C00F03D
:1057B00069802DE9F04B4FF00006002B1FBFB3FAB4
:1057C00083F503FA05F424FA05F65E4012BF16438A
:1057D000B2FA82F502FA05F4C5F120051EBF22FADD
:1057E00005FC44EA0C04203556EA044C4FEA144404
:1057F00018BF641C4FF000084FF00009904271EB95
:10580000030C39D3002919BFB1FA81F701FA07F661
:10581000B0FA80F700FA07F6C7F120071EBF20FA9A
:1058200007FC46EA0C062037B6FBF4FCA7EB05079D
:10583000103F07F01F0BCBF120060CFA0BFB2CFAE4
:1058400006F644BFB3460026202FA4BF5E464FF0A5
:10585000000B5BEA060C08BF4FF0010B19EB0B09BC
:10586000ABFB027C48EB0608C01B06FB02CC0BFB23
:1058700003CC71EB0C01C1E70B460246414648469A
:10588000BDE8F08B13B54FF000004FF00001AFF30F
:105890000080BDE81C4070470446AFF300802046FE
:1058A000FAF78EFC7047000001491820ABBEFEE7F6
:1058B00026000200012181404FF0005010F8352FE2
:1058C0008A4302707047012181404FF0005010F868
:1058D000352F0A430270704710B50B480A4A00780A
:1058E00051789278012803D8012901D8012A09D9D1
:1058F000064B1B6893F8E337FA2B01D1FEF70AFB3E
:10590000012010BD002010BD87021000E002100031
:10591000441D0A5D3F1E1D1D06080708220F052FA6
:10592000200F0F0F020404041108031810080808C0
:10593000000202020904020C08040404000101012F
:105940005A280D7B54282828090B090B2D14073ED3
:105950002A14141404060506170A041F150A0A0A55
:10596000010303030C0502100B05050500020202EA
:105970000001010201020203010202030203030407
:10598000000000001B0000802D0000803600000099
:10599000410000805A0000006C0000007700008089
:1059A0009900008082000000B4000000AF00008079
:1059B000D8000000C3000080F5000080EE00000069
:1059C0002901008032010000040100001F01008055
:1059D0006801000073010080450100805E01000045
:1059E000B0010000AB0100809D0100808601000035
:1059F000F1010080EA010000DC010000C701008025
:105A00004902008052020000640200007F02008010
:105A10000802000013020080250200803E02000000
:105A2000D0020000CB020080FD020080E6020000F0
:105A3000910200808A020000BC020000A7020080E0
:105A4000600300007B0300804D03008056030000CC
:105A5000210300803A0300000C03000017030080BC
:105A6000F9030080E2030000D4030000CF030080AC
:105A7000B8030000A3030080950300808E0300009C
:105A80008904008092040000A4040000BF04008088
:105A9000C8040000D3040080E5040080FE04000078
:105AA000100400000B0400803D0400802604000068
:105AB000510400804A0400007C0400006704008058
:105AC000A0050000BB0500808D0500809605000044
:105AD000E1050080FA050000CC050000D705008034
:105AE0003905008022050000140500000F05008024
:105AF0007805000063050080550500804E05000014
:105B0000C0060000DB060080ED060080F6060000FF
:105B1000810600809A060000AC060000B7060080EF
:105B20005906008042060000740600006F060080DF
:105B30001806000003060080350600802E060000CF
:105B4000E9070080F2070000C4070000DF070080BB
:105B5000A8070000B3070080850700809E070000AB
:105B6000700700006B0700805D070080460700009B
:105B7000310700802A0700001C070000070700808B
:105B80000909008012090000240900003F09008073
:105B90004809000053090080650900807E09000063
:105BA000900900008B090080BD090080A609000053
:105BB000D1090080CA090000FC090000E709008043
:105BC000200800003B0800800D0800801608000037
:105BD000610800807A0800004C0800005708008027
:105BE000B9080080A2080000940800008F08008017
:105BF000F8080000E3080080D5080080CE08000007
:105C0000400B00005B0B00806D0B0080760B0000EA
:105C1000010B00801A0B00002C0B0000370B0080DA
:105C2000D90B0080C20B0000F40B0000EF0B0080CA
:105C3000980B0000830B0080B50B0080AE0B0000BA
:105C4000690A0080720A0000440A00005F0A0080AE
:105C5000280A0000330A0080050A00801E0A00009E
:105C6000F00A0000EB0A0080DD0A0080C60A00008E
:105C7000B10A0080AA0A00009C0A0000870A00807E
:105C8000800D00009B0D0080AD0D0080B60D000062
:105C9000C10D0080DA0D0000EC0D0000F70D008052
:105CA000190D0080020D0000340D00002F0D008042
:105CB000580D0000430D0080750D00806E0D000032
:105CC000A90C0080B20C0000840C00009F0C008026
:105CD000E80C0000F30C0080C50C0080DE0C000016
:105CE000300C00002B0C00801D0C0080060C000006
:105CF000710C00806A0C00005C0C0000470C0080F6
:105D0000C90F0080D20F0000E40F0000FF0F0080D9
:105D1000880F0000930F0080A50F0080BE0F0000C9
:105D2000500F00004B0F00807D0F0080660F0000B9
:105D3000110F00800A0F00003C0F0000270F0080A9
:105D4000E00E0000FB0E0080CD0E0080D60E00009D
:105D5000A10E0080BA0E00008C0E0000970E00808D
:105D6000790E0080620E0000540E00004F0E00807D
:105D7000380E0000230E0080150E00800E0E00006D
:105D80004B38000087380000F53A0000EF3A000079
:105D90009D3600009D3600009D360000C53700008E
:105DA0009D360000A93900009B38000049390000E9
:105DB000CB380000273900000F3B0000493B0000B2
:105DC000673700006B370000FB3A0000DF39000046
:105DD0009D3600009B3700009D36000037380000DC
:105DE000413800009D3600000B3B00009D3600004E
:105DF0005B3B0000D13B0000E93700001F3800008A
:105E00009D3600009D3600009D3600009D36000046
:105E10009D3600009D3600009D3600009D36000036
:105E20009D3600009D3600009D3600009D36000026
:105E30009D3600009D3600009D3600009D36000016
:105E4000046C00080000047C034300011878010082
:105E50001A604002400C03000782000C0D00000095
:105E600000000000005F000005000000A405100015
:105E700000040000151B00000000000002000000EC
:105E800001000000545F000004000000A40910009D
:105E900040060000B12200000000000002000000E7
:105EA00002000000845F000003000000E40F100007
:105EB000000800006935000000000000020000003A
:105EC00003000000205F000002000000E417100043
:105ED00000010000153C000000000000020000006E
:105EE00004000000305F000001000000E418100012
:105EF0008000000061360000000000000200000089
:105F000000000000285F0000010000000100000008
:105F1000605F000001000000020000006C5F0000F4
:105F200001000000030000003C5F000001000000D1
:105F3000000000000C5F000001000000485F00004E
:105F4000020000007C5F000003000000185F0000FA
:105F500054736B5F5353766300000000456C665FBB
:105F60005373766300000000456C665F436D640008
:105F700054736B5F436D640053656D5F41666500EC
:105F800054736B5F49646C650000000053656D5F7E
:105F90004D54427566660000456C665F5363616EE2
:105FA0000000000054736B5F5363616E00000000DB
:105FB00053656D5F4576744669666F0053656D5F26
:105FC00043616C69624672616D657300456C665F22
:105FD0004D74000054736B5F4D740000BC5F000093
:105FE00000021000180100001C010000D460000035
:105FF00000FC1000040100001C010000D46000003F
:1060000018031000EC1B0000380100000000000025
:106010000000000000000000000000000000000080
:106020000000000000000000000000000000000070
:106030000000000000000000000000000000000060
:106040000000000000000000000000000000000050
:106050000000000000000000000000000000000040
:106060000000000000000000000000000000000030
:106070000000000000000000000000000000000020
:106080000000000000000000000000000000000010
:106090000000000000000000000000000000000000
:1060A00000000000000000000000000000000000F0
:1060B00000000000000000000000000000000000E0
:1060C00000000000000000000000000000000000D0
:1060D00000000000000000000000000000000000C0
:1060E00000000000000000000000000000F001209F
:1060F0004C00012000000000000000000000000033
:10610000000000000000000000000000000000008F
:10611000000000000000000000000000000000007F
:106120000000000030B572B601250D4C256000233B
:106130006A07012910D082F86B3000F03F0082F826
:106140006A000848056001680029FCD105481C3038
:106150000360236062B630BD402182F86B10ECE72B
:10616000401B00225C0D0022FCB54FF00052D020F5
:1061700082F8C3002B4F386848B140F29B70D0843E
:106180004520A2F85200A2F85200FA2008E040F29E
:106190002F30D0843120A2F85200A2F85200BC2047
:1061A000402482F82040442582F8205000234FF4F8
:1061B0009676CDE90063194605E00099491E0091E5
:1061C0000199491C01918142F7D30FE082F82040E8
:1061D00082F82050CDE90063194605E00099491E78
:1061E00000910199491C01918142F7D392F8201046
:1061F000C906EBD482F8C330386828B141F2984020
:10620000D08440F2572004E041F22C00D08440F2C8
:10621000C110A2F85200A2F852004C2082F82000CF
:10622000FCBD0000DC040022A50E10000100004AA5
:106230000705194D01FF961F0C100F23DC052C01DB
:10624000DC052C0100000000D00700000000000069
:106250000000030932000000000000000000000000
:1062600000000F010A05002C012C01FA0000009625
:106270006464005E01F401C80094021405F6094844
:106280000DD20F0000000032200300910032000008
:1062900000011A0503021A0401013F024400000331
:1062A00000010080000000001E014006960008006A
:1062B000E50064001F04000010000001980A0B6450
:1062C0000000000000000000030010051014000092
:1062D00000000000000000000000024B03320064D8
:1062E000283C401F401F32A00FB80BA00FB80B2D49
:1062F0000D64640000000000003C000045960000B2
:10630000050C000003010000060900004080004069
:1063100080000000000000000000000000000000FD
:10632000000000000000000000000000000000006D
:10633000000000000000000000000000ECECECECAD
:10634000ECEC000000000000000000002D2D2D2DC1
:106350002D2D00003C3C3C3C3C3C000023232323EF
:10636000232300000A010F190F1400000000000091
:10637000000000000000000000000000000000001D
:10638000000000000000000000000000000000000D
:1063900000000000000000000000000000000000FD
:1063A00000000000000000000000000000000000ED
:106A00000000000000000000000002000000000084
:106A1000000000000E100000000000000000000058
:0C6A200000000000D00A9F25E321170DA4
:00000001FF
